:1000000012C0189518951895189518951895189563
:100010001895189518951895189518951895189578
:100020001895189518958FED8DBFC0ECE0EC4E2E0D
:10003000DD275D2EEEE7F0E0A0E6B0E0A89584B7FE
:10004000082E877F84BF88E1992781BD91BD8827CD
:100050008D933197E9F7C4D266248FE087BB80E0A7
:1000600088BB8FEF81BB80E082BB84E690E02CD31D
:100070008CE0FED2BF98A7E69C9197FF04C0B79989
:100080000EC09F779C93B79B0AC088E29F939927E5
:100090001BD39F91B79B03C090689C9330D286D2AC
:1000A000EEE3F7E07BD280D2EEE4F7E077D2E2E055
:1000B000F0E08DD2E9E0F0E0A6E691E039D30091DE
:1000C00066000E3C08F004C085B7816285BF889544
:1000D00080E080936400A1E60AD380E0809363000F
:1000E00080E08093650062D2EEE5F7E057D288E0C9
:1000F00087BB80E788BB8AE090E0E6D281E080930E
:100100006000A6E30C9105FB81E00EF480E08F9384
:10011000A6E30C9106FB81E00EF480E09F91892319
:10012000882309F401C00CD182E080936000A6E32B
:100130000C9104FB81E00EF480E08F93A6E30C9118
:1001400005FB81E00EF480E09F918923882309F468
:1001500001C0F6D083E080936000A6E30C9104FB1D
:1001600081E00EF480E08F93A6E30C9106FB81E022
:100170000EF480E09F918923882309F401C0E0D028
:1001800080E187BB88E688BB8AE090E09DD284E06E
:1001900080936000A6E30C9105FB81E00EF480E003
:1001A0008F93A6E30C9106FB81E00EF480E09F9113
:1001B0008923882309F401C0C3D085E080936000BF
:1001C000A6E30C9105FB81E00EF480E08F93A6E39B
:1001D0000C9106FB81E00EF080E09F91892388233B
:1001E00009F401C0ADD086E080936000A6E30C91D5
:1001F00005FB81E00EF080E08F93A6E30C9106FBF7
:1002000081E00EF480E09F918923882309F401C0E6
:1002100097D080E287BB88E588BB8AE090E054D223
:1002200087E080936000A6E30C9104FB81E00EF070
:1002300080E08F93A6E30C9106FB81E00EF480E052
:100240009F918923882309F401C07AD088E08093A4
:100250006000A6E30C9104FB81E00EF480E08F9334
:10026000A6E30C9106FB81E00EF080E09F918923CC
:10027000882309F401C064D089E080936000A6E37C
:100280000C9104FB81E00EF480E08F93A6E30C91C7
:1002900006FB81E00EF480E09F918923882309F416
:1002A00001C04ED080E487BB88E388BB8AE090E041
:1002B0000BD28BE080936000A6E30C9104FB81E0FD
:1002C0000EF080E08F93A6E30C9105FB81E00EF425
:1002D00080E09F918923882309F401C031D08AE00E
:1002E00080936000A6E30C9104FB81E00EF480E0B3
:1002F0008F93A6E30C9105FB81E00EF480E09F91C3
:100300008923882309F401C01BD08CE0809360000E
:10031000A6E30C9104FB81E00EF480E08F93A6E34A
:100320000C9105FB81E00EF080E09F9189238823EA
:1003300009F401C005D08AE090E0C6D1D8CE95CEB0
:10034000939A84E690E0C0D1939884E690E0BCD183
:1003500000916400013009F001C02AC000916400DE
:10036000023009F001C047C0009160000B3009F075
:100370000CC01CD1ECE6F7E011D1A4E68C918F5FA4
:100380008C9380E080936300B2CE009160000C30CB
:1003900009F00DC0EAE0F0E0A4E1C9D1A1E60D91B9
:1003A0001C910417150709F001C088C065C036C04C
:1003B000009160000C3009F01DC0EAE0F0E0A4E11B
:1003C000B6D1A1E60D911C910417150709F401C0DF
:1003D00053C0A1E68CD180E08093630080E08093DD
:1003E0006500A4E68C918F5F8C93E0D0ECE7F7E09A
:1003F000D5D07DCE13C0009160000C3009F00EC046
:10040000EAE0F0E0A1E67BE781D1D0D0ECE8F7E0CC
:10041000C5D043D0E2E0F0E0DAD04CCEA3E68C9138
:100420008F5F8C930091630044E0040FA5E60C936A
:100430008FEBA5E61C91C9D0ECE9F7E0AFD00091B5
:100440006300083010F009F001C001C015C0A1E63A
:100450000D911C914AE050E08ED0A1E60D931C93C3
:10046000A1E60D911C91A0E64D915527040F151F93
:10047000A1E60D931C93089599D0EEE9F7E08ED094
:10048000939AE3E0F0E0A3D093988ED0EEE3F7E008
:1004900085D0E4E1F0E09BD00DCE84E690E014D16D
:1004A000939A88EC90E010D1939888EC90E00CD16E
:1004B000939A88EC90E008D1939808958091660013
:1004C000815080936600E9E0F0E0A6E691E07BE7EA
:1004D0001ED16CD0ECE8F7E061D0DFDF65D0ECEA4C
:1004E000F7E05CD08CE291E0EFD0949AE1E0F0E0AC
:1004F0006ED094985BD0E1E0F0E069D0DBCDE1E034
:10050000F0E065D0B79901C014C0EAE0F0E002ED78
:1005100014E0A0E1BB277BE7F9D0BFDF47D0EAEBCF
:10052000F7E03CD041D0EAECF7E038D0E4E0F0E08E
:100530004ED0089504D01FD000FC0CD008950024A4
:10054000E89457FF02C009D0689400F80BD010F867
:100550000124089502D009D00895509540954F5F29
:100560005F4F0895E89417FF0895009510950F5F69
:100570001F4F68940895752F642F55274427FF93C4
:10058000F1E1889405C010F4460F571F5695479522
:1005900017950795FA95B9F7FF910895A4D0802D86
:1005A00011F060D0FBCF089580EC62C081E060D094
:1005B00014D080E85DC08FE7213039F08FEB223016
:1005C00021F08FE8233009F08FEC810F51C088EEC5
:1005D00093E07AD03197D9F7089583E0992774C0D2
:1005E0008AEF90E071D0BB9ABA9AB99AB89A8E9A6B
:1005F0008D9A959885E090E067D09698C398C298B8
:10060000C19AC09A969AEF93FF93E5E1F0E050D03B
:10061000FF91EF91969855D0969AEF93FF93E5E16D
:10062000F0E046D0FF91EF9196984BD0969AEF93D9
:10063000FF93E5E1F0E03CD0FF91EF91969841D037
:10064000C098969AEF93FF93E5E1F0E031D0FF91E7
:10065000EF91969836D088E20BD08EE009D086E0F4
:1006600007D00895959A829505D004D02AD0089590
:100670009598F9CF859510F4C09A01C0C0988595DA
:1006800010F4C19A01C0C198859510F4C29A01C0B6
:10069000C298859510F4C39A01C0C398969AEF93B7
:1006A000FF93E5E1F0E004D0FF91EF919698089573
:1006B0003197F1F70895689462F80895E89462F824
:1006C000089581E090E000C0EF93FF93EE27E82BC0
:1006D000E92B31F0EAEFF0E03197F1F70197D1F72C
:1006E000FF91EF910895C89531960020089582E01A
:1006F00001C084E099279D938A95E9F70895E199CF
:10070000FECFEEBB3196089591E001C092E07B37B9
:1007100051F47FB7F894F3DF8D918DBBE29AE19AA3
:100720009A95C9F77FBF7727089591E001C092E0BD
:10073000E6DFE09A8DB38D939A95D1F708955757D8
:10074000572E4156522E344D472E434F4D00436F86
:1007500064654C6F636B415652202D20520020205F
:1007600020456E74657220636F64650020456E7469
:100770006572206F6C6420636F64650020456E7441
:100780006572206E657720636F64650020436F6437
:100790006520616363657074656400002A00202031
:1007A00020436F64652077726F6E670020202020E1
:1007B000556E6C6F636B656400002020496E697430
:1007C00069616C20636F646500002020202020692F
:0A07D0007320202031323334000082
:00000001FF
